:1000000010C02AC029C028C027C026C025C024C0CF
:1000100023C022C021C027C01FC01EC01DC01CC0DD
:100020001BC011241FBECFE5D2E0DEBFCDBF10E064
:10003000A0E6B0E0ECE4F1E002C005900D92A0363D
:10004000B107D9F710E0A0E6B0E001C01D92A936D3
:10005000B107E1F704D078C0D3CF0895089557D001
:10006000FCDFFCDFFECF1F920F920FB60F92112420
:100070002F933F934F935F936F937F938F939F93B0
:10008000AF93BF932091640030916500409166006A
:100090005091670070916800DA01C9014096A11D76
:1000A000B11D672F605D6D3730F06D57DA01C90102
:1000B0004196A11DB11D60936800809364009093E8
:1000C0006500A0936600B0936700809160009091F6
:1000D0006100A0916200B09163000196A11DB11D65
:1000E0008093600090936100A0936200B0936300DE
:1000F000BF91AF919F918F917F916F915F914F9140
:100100003F912F910F900FBE0F901F9018957894EC
:1001100080B7826080BF80B7816080BF83B7826014
:1001200083BF83B7816083BF89B7816089BF8EB584
:1001300082608EBD8EB581608EBD8FB581608FBDB2
:0C014000319A309A379A0895F894FFCF56
:00000001FF
